:020000040000FA
:020000008C284A
:08000800A000030E8301A1001A
:100010000A08A2008A010C1C3A280C10400810396A
:10002000031914281F141F15B00AB00A3C303006FB
:10003000031D3A280030B000B20A3C303206031DDE
:100040003A280030B200B10A18303106031D3A28B0
:100050000030B100B30A6823013E3306031D3A287D
:100060000130B300B40A0D303406031D3A280130C4
:10007000B400B50A06081039031949284008103998
:10008000031D49281030C0000030C100CE2150248B
:100090002424060810390319C0000C1F6A280C1309
:1000A0001F104608C5000130C6001E08C7003F08E3
:1000B0004702031CC60146084506031D6A28450879
:1000C000440603196A284508C40003196928F9225F
:1000D0006A2820230B1C7E280B10D6213808031D0C
:1000E000FB2106082039390603197E280608203925
:1000F000B90006082039031D7E2891224008031903
:100100008228CD2085018601870122088A00210EE0
:100110008300A00E200E090083160E309F0083126C
:1001200041309F0083168230810001308500F0301D
:10013000860000308700831286010030B1009014E1
:10014000901510129012101510140130B300B40065
:10015000B5000030B100B200B0004016C301C401C8
:10016000C501C6015030C8001224D2005130C80069
:100170001224D1005230C8001224BF00D3215024D1
:1001800024240C100C1383160C140C1783120B1759
:100190008B158B178B176300CA284108023A031985
:1001A00080294108863A03193E293B243308A500DB
:1001B000AD2344242E309E243408A500AD234424CE
:1001C0002E309E243508A500AD2344240B3038245E
:1001D0003108A500AD2344243A309E243208A500FE
:1001E000AD2344243E244308A50008308823C800DA
:1001F0000830BB001E244108013A031D1129D422F6
:1002000049303824F6309E2420309E246008A50012
:10021000AD2344242E309E246108A500AD23442440
:100220001D29493038244408A50008308823403E61
:10023000C8000730BB001E241D290C308D24410846
:10024000013A031D78294030C2003929410880391C
:100250000319CD2941087F39C2000130C2020330A1
:10026000A50042088823C200183903193929023031
:10027000C207420838240F308D24CD293B24533047
:100280009E2463309E2468309E2477309E246530FF
:100290009E246C309E246C309E2465309E24203039
:1002A0009E2453309E2470309E2465309E246530F9
:1002B0009E2464309E243E2453309E246F309E241E
:1002C0006C309E246C309E243A309E243F08A5005A
:1002D000AD23492420309E2449309E2473309E242F
:1002E00074309E243A309E244708A500AD2349244B
:1002F0004108863A031D26294530C2003929CD29F7
:100300000C308D243B245308A500AD2344242E300B
:100310009E245408A500AD2344242E309E24550865
:10032000A500AD23442420309E245C08A50008309D
:100330008823C8000430BB001E2420309E245008AF
:10034000A500AD2344243E245608A500AD23442433
:100350003A309E245708A500AD2344242D309E2416
:100360005808A500AD2344243A309E245908A5001E
:10037000AD2344245A08A500AD2344243A309E24DA
:100380005B08A500AD2344244B30382420309E2444
:100390000E3038240F308D24CD290800060820396E
:1003A000B900861A08008130C10008003608B7007D
:1003B0000608B6000630BC00B60CBC0BDC290330C6
:1003C000B605370836060319F82901303606031931
:1003D000F829023036060319F8293708360601399C
:1003E0000319F529FF30B80008000130B8000800F3
:1003F0000030B800080002304106031D102A3808FA
:10040000D007B81F082A5108FF3E50060319D00A2A
:10041000B81B0F2A5208013E50060319D003A72229
:1004200001304106031D222A3808C307FF30430666
:10043000031D1C2A0330C30004304306031D222A77
:100440000030C30081304106031D342A3808B30749
:1004500000303306031D2E2A1F30B3002030330630
:10046000031D342A0130B30082304106031D462AA1
:100470003808B40700303406031D402A0C30B4009D
:100480000D303406031D462A0130B4008330410686
:10049000031D582A3808B507FF303506031D522AB8
:1004A0001F30B50020303506031D582A0030B50036
:1004B00084304106031D6A2A3808B107FF3031062F
:1004C000031D642A1730B10018303106031D6A2A53
:1004D0000030B10085304106031D7E2A3808B2077E
:1004E0003008B006FF303206031D782A3B30B200D8
:1004F0003C303206031D7E2A0030B20086304106B1
:10050000031D902A3808BF07FF303F06031D8A2AC3
:10051000FE30BF00FF303F06031D902A0030BF00B1
:100520000800C10A033041060319C10187304106A2
:10053000031D9F2AC1015230C8003F08FC2302302E
:100540004106031DA62A5208D000A72208001C302D
:10055000C9005008CA00E6233A23C90AE6235423F7
:100560005808D6005908D700C90AE6235423C90AF7
:10057000E6236723440801390319C82A50085206A4
:10058000031DC82A4308DC003108D8003208D9000E
:1005900056085802DA0057085902DB00DB1FD32A3D
:1005A0003C30DB07DA030800E001E1015208D0002B
:1005B0005008510603190800A72233085306031DEB
:1005C000080034085406031D080035085506031DAD
:1005D000080043085C06031DF72A5B08E1075A0878
:1005E000E0073C306102031CF72AE102E00AD00375
:1005F000D82A5208031D032B5106031D032B01307B
:10060000D200D100082BD20A520851060319D10A90
:100610005030C8005208FC235130C8005108FC2358
:100620005208CA001C30C9002A23C823C90A47231C
:10063000C823CC01CB01C90AC823C90AC8230800B2
:100640005208CA001E30C9004723C823C90A6423C0
:10065000C82308003508CB00CC00CC0EF030CC0508
:1006600034080F39CC04CB0D2030CB0533081F39AB
:10067000CB0408004C08D400D500D50E0F30D405AB
:10068000D5054B08D3001F30CB1A55160800320889
:100690003F39CC0031081F39CB0043184C17C31821
:1006A000CC174319CB1608004C08D9003F30D905A8
:1006B0004B08D8001F30D805DC014C1B5C14CC1B48
:1006C000DC14CB1A5C150800CB01CC010800080033
:1006D00002303406031D742B033035050319722BC9
:1006E0001C3008001D300800043034060319862B26
:1006F000063034060319862B093034060319862B7D
:100700000B3034060319862B1F3008001E300800FA
:10071000BA00031D8D2B0030A5002508BA0303196C
:10072000932BA5078E2B250808002308A50724086E
:100730000318240FA6070800A8012308A502031820
:10074000A52B0130A602031C28142408A602031CB2
:10075000281403102818031408000330A400E830FC
:10076000A300C023A900A4016430A300C023AB00F0
:10077000A4010A30A300C023AA002508AC00080089
:10078000A701A70A9C23031CC12B9523270308005C
:100790004908031783128F0003134A0803178D00BB
:1007A00003134B0803178E0003134C0803178C0028
:1007B00083168C170C158B1355308D00AA308D00C5
:1007C0008C1400000000031383120800490803176B
:1007D00083128F0003134A0803178D0083168C17AA
:1007E0000C140000000083120C080313CC00031744
:1007F0000E080313CB0008000D12031783128C00A0
:100800000313480803178D0083168C130C158B13E4
:1008100055308D00AA308D008C14031383120D1EE9
:100820000F2C08004808031783128D0083168C13C1
:100830000C1483120C0883120313080012249E2444
:10084000C80ABB0B1E2C08003B241030BB00203014
:10085000C8001E243E241030BB003030C8001E24C7
:100860000430A500FA30BD00B224A50B322C0800DC
:1008700080388D24080001308D2408004030382451
:10088000080030389E2408002A0841242C084124FE
:1008900008002B0841242A0841242C084124080080
:1008A000FF30BD00B224303087000614000006106F
:1008B0003230BD00B22430306E2430306E2420300F
:1008C0006E2401308D2428308D2408308D2406308C
:1008D0008D2403308D240C308D24080087000614ED
:1008E000000006100A30BD00B22408008316F03064
:1008F0008704831206118614061400000708AD0051
:1009000006100000061400000610AD1B7A2C86109D
:1009100083160F30870583120800AE0076242E0858
:10092000F03987000614000006102E0EF0398700FB
:100930000614000006100F3087050800AE0076246C
:100940002E08F039870006150614000006102E0E3A
:10095000F0398700061506140000061006110F3046
:10096000870508006430BE000000000000000000A1
:10097000000000000000BE0BB42CBD0BB22C0034F4
:02400E00313F40
:1042000054004F00420049004B00200020002000D5
:1042100042004F00520043004800490020002000A7
:1042200054004B002B0042005000200020002000D2
:1042300047004100530054002000200020002000CF
:1042400054004F00420049004B007300200046001C
:104250006C0069006700680074004C006F00670024
:10426000280063002900300037002F0032003000A2
:10427000300033002000560031002E0030003100A5
:1042800020005000410052004B0045004E0020002D
:1042900046004C0049004500470045004E00200004
:1042A00000000000500000000000000000000000BE
:00000001FF
